:107800000C945D3C0C94953C0C947A3C0C947A3C22
:107810000C947A3C0C947A3C0C947A3C0C947A3C10
:107820000C947A3C0C947A3C0C947A3C0C947A3C00
:107830000C947A3C0C947A3C0C947A3C0C947A3CF0
:107840000C947A3C0C947A3C0C947A3C0C947A3CE0
:107850000C947A3C0C947A3C0C947A3C0C947A3CD0
:107860000C947A3C0C947A3C040309041C037700C2
:10787000770077002E0066006900730063006800DF
:107880006C002E00640065000E035500530042009A
:1078900061007300700012011001FF000008C016A3
:1078A000DC05020101020001090212000101008051
:1078B000FA09040000000000000011241FBECFEFF1
:1078C000D8E0DEBFCDBF11E0A0E0B1E0ECEDFFE716
:1078D00002C005900D92A630B107D9F711E0A6E0DD
:1078E000B1E001C01D92AC33B107E1F70E94CF3D7A
:1078F0000C94EC3F0C94003CA82FB92F80E090E052
:1079000041E050EA609530E009C02D9182279795BB
:10791000879510F084279527305EC8F36F5FA8F332
:107920000895EADF8D939D930895CF93CFB7CF93BA
:10793000C3954F9BE9F74F9B09C04F9B07C04F9BD7
:1079400005C04F9B03C04F9B01C0A1C0DF93C091F6
:107950001F01DD27CA5DDE4F4F9B02C0DF91EBCFD9
:107960002F930F931F9309B12FEF07FB20F94F932C
:107970003F9319B14FEF012707FB21F93BE031C0DD
:107980004E7F012F19B1216028C0102F4D7F22603A
:10799000000009B129C04B7F2460012F000019B1FC
:1079A0002BC019B1477F28602AC04F7E09B12061E2
:1079B0002CC04F7D19B120622FC04F7B09B12064CC
:1079C00032C0422709B149934FEF0000102717FB3F
:1079D00020F919B11478C9F1297F91F2012707FB29
:1079E00021F909B1237F89F2315058F1102717FB93
:1079F00022F919B1277E79F2012707FB23F92F7CA1
:107A000081F209B1102717FB24F92F7971F200C018
:107A100019B1012707FB25F92F7359F200C009B1ED
:107A2000102717FB26F9223040F200C019B10127B8
:107A300007FB27F9243028F64F77206819B100009A
:107A4000F9CF11E01CBB002717C03B503195C31B79
:107A5000D04011E01CBB0881033CE9F00B34D9F0A5
:107A600020911D011981110F1213EDCF093641F13B
:107A70000D3211F0013E39F7009324013F914F91EF
:107A80001F910F912F91DF91CCB3C0FD51CFCF91BA
:107A9000CFBFCF91189520912401222379F3109123
:107AA0002201112311F5343012F130932201209379
:107AB0001E0110911F013BE0311B30931F0117C0C5
:107AC0000091220101308CF40AE53091000134FD6F
:107AD00010C000930001C2E1D1E00FC02795A8F4C7
:107AE0005150A9F4220F0000F9CF4AE503C042ED3E
:107AF00001C0432FC4E1D0E032E01AB114685F9AAC
:107B00001AB90BB120E414E85F93012756E00BB9D2
:107B1000279520F4515021F4220FF9CF012756E088
:107B200000003B5A0BB9D0F2279528F4515029F4A4
:107B3000220F0000F9CF012756E027950BB920F45A
:107B4000515021F4220FF9CF012756E02991332318
:107B50000BB921F60B7710912301110FC651D040BC
:107B60000BB911F010931D0111E01CBB00681AB194
:107B70001B77402F4B775F9100C000C00BB91AB93B
:107B80004BB97CCF1BB8F8941DBA1092690081E004
:107B900085BF15BEE0911001F091110109952F925A
:107BA0003F924F925F926F927F928F929F92AF928D
:107BB000BF92CF92DF92EF92FF920F931F93CF93DA
:107BC000DF9388E10FB6F894809360001092600014
:107BD0000FBE5F9A04B601FEE7C114BE81E085BF07
:107BE00082E085BF4F99E0C18091690083608093F6
:107BF0006900E89A4F9BFECF579878946CE0262E48
:107C0000312C03E058E8C52E58E7D52E4CE6A42EBB
:107C100048E7B42E38E6832E38E7932E28EA622E02
:107C200028E7722E96E9492E98E7592E87E0E82E2C
:107C300081E0F82E90912201935097FD29C1809107
:107C40001F01E101C81BD109CA5DDE4F80911E01F1
:107C50008D3209F0C1C0983009F018C123EC20938F
:107C600012018AE58093000110920B013881832F65
:107C700080762981882309F444C0F0922101E092A2
:107C800020012330D9F49B818C812A81203339F45F
:107C90008370E82FF0E0EE5FFE4F80810BC0203A4A
:107CA00019F40E94D63F06C0203C19F46D810E9451
:107CB000DE3F80E080930A0194E07EC0253011F41D
:107CC00091E07AC0822F84508630A0F48A819B8113
:107CD00090930D0180930C01293009F46CC09E81B2
:107CE00090930E018D81827080930F0137FD68C0E3
:107CF0002FEF67C0223009F05EC0E1E0E09306019B
:107D00005AC08A8110921B01222331F410921C0167
:107D10002BE131E092E04AC0253019F48093230131
:107D200042C0263081F58B81813029F450922101A7
:107D30004092200106C0823031F47092210160929D
:107D4000200192E11CC08330C9F48A81882331F478
:107D5000909221018092200194E011C0813031F491
:107D6000B0922101A09220019CE109C0823031F43F
:107D7000D0922101C09220019EE001C090E0F0E489
:107D8000F0930B0119C0283019F425E231E009C045
:107D9000293019F48093250106C02A3021F42BE103
:107DA00031E091E003C02BE131E090E0309321011C
:107DB0002093200101C090E08F81882331F008C01A
:107DC000292F80E880930B0104C02E81291708F029
:107DD000292F209301015AC080910B0187FF56C0C3
:107DE00080910E01592F891708F4582F851B809315
:107DF0000E0160E0882309F461E070910F01E091C9
:107E00000C01F0910D0140E036C0CF018F779070EA
:107E1000892B41F4F89400935700E895789407B6BD
:107E200000FCFDCF4E5FF8948991999121E00C01FF
:107E300020935700E895112478949F012E5F3F4FBF
:107E4000C9018F779070892B31F0662399F045171F
:107E500088F0772379F0F89485E080935700E895CF
:107E6000789407B600FCFDCFF894E1E1E093570069
:107E7000E8957894F901451708F4C7CFF0930D0100
:107E8000E0930C01662311F010920101109222017F
:107E90008091000184FF79C0809101018F3F09F436
:107EA00074C0182F893008F018E0811B80930101FD
:107EB0008091120198E8892780931201112309F417
:107EC00051C080910B0187FF1EC080910E01811768
:107ED00008F4182F811B80930E01A0910C01B09122
:107EE0000D01AD01C3E1D1E0212F30E0B9016C0FEC
:107EF0007D1F05C0FA01849189934F5F5F4FC617BC
:107F0000D707C1F727C0209120013091210186FFBA
:107F10000DC0A3E1B1E080E090E0F901E80FF91FA6
:107F2000E491ED9301961817C1F708C0D901912F7C
:107F3000E3E1F1E08D9181939150E1F71150812FB0
:107F400090E01F5F0196820F931F90932101809311
:107F5000200108C02A0F3B1F30930D0120930C0114
:107F6000193068F483E191E0612F0E94913C612F08
:107F70006C5F6C3041F08FEF8093010104C08FEF94
:107F8000809301016EE16093000194E189B18478EE
:107F900031F49150D9F71092230110921D01809174
:107FA0000601882309F446CE0E94C23DF999FECF0E
:107FB00092BD81BDF89A992780B50895262FF99929
:107FC000FECF1FBA92BD81BD20BD0FB6F894FA9ABC
:0C7FD000F99A0FBE01960895F894FFCFB7
:067FDC005AFF1E950F0084
:040000030000780081
:00000001FF
